:020000040000FA
:10000000831607309C0001309B0000309F00811355
:100010000030860013308500831201309F000030CD
:100020008B00860185011E21C31033213E20BD1F98
:10003000C82033203E20BD1B1A28872043181A28C9
:10004000C206031D3028C200B70AB71F1A283F3E58
:1000500062210130420603193320B7013A201A28E1
:10006000C200B7011A2801305F2107305F218F30AD
:100070005F2108003E20BD1F3A280800831680300B
:1000800086001230850002309B00831209309F00E9
:1000900006130514C31C4E2882305F216320BD0067
:1000A0008316403086001130850001309B0083129A
:1000B00001309F0086138514C31C6028C2305F2165
:1000C0006320BE0008001F151F1964281E08B90010
:1000D000C31C0800BC00BA01BA0A6430BC02031891
:1000E0006C286430BC07BA03BB01BB0A0A30BC02EF
:1000F000031875280A30BC07BB033A0861213B0886
:1001000061213C0861212030622139080800431038
:100110003E08BF0020308400A720BE003D08BF007D
:100120002A308400A720BD00431808002908C10018
:10013000C001C10C031C9E283E08C0070310BE0D61
:100140004108031D992840083D07013E0800C420CE
:10015000031C0034C420031C0134C420031C0234DB
:10016000C420031C0334C420031C0434C420031C17
:100170000534C420031C0634C420031C0734C420E7
:10018000031C0834431408000008840A3F020800D6
:10019000C314B701C401203084003E20C6305F2163
:1001A000B70A370807396121371FCD283E08C40236
:1001B0000318E328B7018000C400840A3A203E20D7
:1001C000BD1BDF28CD28B701B801C4012A30840047
:1001D0003E20C6305F21B70A370807396121371F33
:1001E000E8283D08C4020318FF28B7018000C400B6
:1001F000840AB80A3A203E20BD1BFB28E828C31019
:100200003808A900831203178D01031320308400DE
:1002100000080E21041B0800840A082903178C001B
:1002200083168C130C1555308D00AA308D008C145C
:100230008C18182983128D0A0313080083120317E0
:100240008D012030840029218000041B0800840ACD
:100250002329031783168C130C14000083120C0837
:100260008D0A0313080020305F2120305F212830E1
:100270005F210E305F2106305F2101305F210230A7
:100280005F2108008511340E0F39860000008515A6
:10029000000000000000851134080F3986000000BE
:1002A000851500000000000085110330B500B60B75
:1002B0005729B50B5729080080305F29C030051138
:0A02C0006329303E0515B400422901
:02400E00413F30
:02401000FC3F73
:104200002200340047005A006C000000000000004B
:10421000000004001A0027003400410000000000E4
:08422000000000000000000096
:00000001FF
